:103800000C942A1C0C94451C0C94451C0C94451CCF
:103810000C94451C0C94451C0C94451C0C94451CA4
:103820000C94451C0C94451C0C94451C0C94451C94
:103830000C94451C0C94451C0C94451C0C94451C84
:103840000C94451C0C94451C0C94451C0C94451C74
:103850000C94451C11241FBECFE5D4E0DEBFCDBFC4
:1038600010E0A0E6B0E0E8E7FDE302C005900D92AD
:10387000A036B107D9F710E0A0E6B0E001C01D9274
:10388000A73EB107E1F70C946F1D0C94001C81E476
:103890000E948C1E86E50E948C1E82E50E948C1E72
:1038A00082E40E948C1E8FE40E948C1E8FE40E9492
:1038B0008C1E84E50E948C1E0895BF92CF92DF92E9
:1038C000EF92FF920F931F93CF93DF938C01B62E4D
:1038D00020E030E0E901CE59DF4F79010894E11C86
:1038E000F11C2017310718F40E94A11E01C08FEFB0
:1038F000888397012038310568F320E030E0C090DC
:10390000E200D090E300E090E400F090E5008CB39A
:103910009927AC014270507081FDF9CF8091E6008B
:10392000853709F07FC086E4B81609F039C041E058
:10393000C2E6D0E08991282F332789919927982FC3
:103940008827282B392B8091E2009091E300090110
:10395000FC0140935700E89511248091E20090917A
:10396000E300A091E400B091E5000296A11DB11D15
:103970008093E2009093E300A093E400B093E5000D
:1039800002501040B9F685E0F60180935700E895A3
:1039900007B600FCFDCF81E180935700E8953FC05A
:1039A00085E4B816E1F58091E2009091E300A091E2
:1039B000E400B091E500B695A7959795879580931B
:1039C000E2009093E300A093E400B093E500F901D6
:1039D000EF59FF4F8091E2008EBB8091E200909101
:1039E000E300A091E400B091E500292F3A2F4B2F7E
:1039F00055272FBB0196A11DB11D8093E200909326
:103A0000E300A093E400B093E500319680818DBB84
:103A1000E29AE19AE199FECF01501040D9F68DE08B
:103A200090E001C0CA01DF91CF911F910F91FF90EB
:103A3000EF90DF90CF90BF9008950F931F93CF9397
:103A4000DF93EC01E199FECF653411F58091E2003E
:103A50008EBB8091E2009091E300A091E400B091D0
:103A6000E500292F3A2F4B2F55272FBB0196A11D7B
:103A7000B11D8093E2009093E300A093E400B09323
:103A8000E500E09A8DB30E948C1E2197F9F622C0C2
:103A9000E091E200F091E30005911491802F0E94E3
:103AA0008C1E812F99270E948C1E8091E20090919C
:103AB000E300A091E400B091E5000296A11DB11DC4
:103AC0008093E2009093E300A093E400B093E500BC
:103AD0002297F1F6DF91CF911F910F910895CFE5D5
:103AE000D4E0DEBFCDBFF89401E005BF82E085BF22
:103AF00060E087E190E00E94821EA098A89A989BBF
:103B000008C0A89805BF15BEE0916000F091610063
:103B100009950E94A11E682F813611F489E5EFC036
:103B2000813439F50E94A11E9927AA27BB278093CB
:103B3000E2009093E300A093E400B093E500EE244C
:103B4000F82E092F1A2F0E94A11E9927AA27BB27FA
:103B5000E82AF92A0A2B1B2BEE0CFF1C001F111F51
:103B6000E092E200F092E3000093E4001093E5009D
:103B700068C0823641F489E50E948C1E80E00E9474
:103B80008C1E80E8BCC0823489F40E94A11E992753
:103B9000182F00270E94A11E9927082B192B0E947D
:103BA000A11E682FC8010E945D1CA9C0873689F438
:103BB0000E94A11E9927182F00270E94A11E992755
:103BC000082B192B0E94A11E682FC8010E941D1DE1
:103BD000A0CF853609F037C08091E600853769F5BA
:103BE0001092E2001092E3001092E4001092E500BF
:103BF00023E08091E2009091E300FC0120935700C4
:103C0000E89507B600FCFDCF8091E2009091E300BB
:103C1000A091E400B091E50080589F4FAF4FBF4F97
:103C20008093E2009093E300A093E400B093E5005A
:103C300080509843A040B040E0F281E1809357006B
:103C4000E8958DE05CC0853451F488E190E028E08F
:103C50000FB6F894A89581BD0FBE21BDF2CF803577
:103C600081F38C3471F3803711F483E548C08634D6
:103C700021F469E080E090E005C0823731F469E02A
:103C800081E090E00E94B51E3AC08E3421F469E0D4
:103C900083E090E0F7CF813521F469E082E090E0A5
:103CA000F1CF843729F485E70E948C1E80E027C07D
:103CB0008857823018F40E94A11EC3CF643529F4BE
:103CC0000E94A11E8093E600BCCF633519F40E94C8
:103CD000471C1FCF663529F480E30E948C1E87E3C2
:103CE0000EC0633741F483E00E948C1E84E90E9479
:103CF0008C1E8EE104C06B3109F40BCF8FE30E9460
:103D00008C1E07CF9C01832F992780BD29B988E19C
:103D10008AB986E880BD089520E030E08CB90FB6FE
:103D200007FE0BC05E990BC02F5F3F4F5E9907C027
:103D300087E220313807C4F302C05E9BFECF5E9A53
:103D4000089580E090E00FB607FE0AC05F990AC0B0
:103D500001965F9907C027E280319207CCF302C039
:103D60005F9BFECF8CB199270895FC0160935700AB
:083D7000C895802D99270895E4
:0400000300003800C1
:00000001FF
